:020000040000FA
:040000008B17F5293C
:08000800FB000308FC000A08DC
:10001000FD008A1183120B1D1628FF0803191228F0
:10002000FF0315287E148B12F9250B117D088A0019
:100030007C088300FB0E7B0E09000008A00008006E
:10004000840A00088403A1001D28840A840A000889
:1000500084038403A20020282008800008002108CF
:10006000840A800084032C282208840A840A8000E1
:10007000840384032F280008A0070800840A0008CE
:100080008403A107031C3B28A00A3B28840A840A96
:10009000000884038403A207031C3E28A10A031D51
:1000A0003E28A00A3E280008A0020800840A000892
:1000B0008403A10203185328A0035328840A840A46
:1000C000000884038403A20203185628A103210A0E
:1000D000031D5628A00356280008200208006C20A3
:1000E000031D0800840A00082102080000082006F9
:1000F000803903196C280314A01B03100800762014
:10010000031D08007228A01BAE280800A01BC328EE
:100110000800A30A031D0800A20A031D0800A10A83
:10012000031D0800A00A0800A01BB528A028A01BDA
:10013000B528A228A01BB528A528A01BB528A9284A
:10014000A0099228A009A1098F28A009A109A20944
:100150008C28A009A109A209A30989287F30A00041
:10016000FF30A100FF30A20008008030A000003066
:10017000A1000030A2000800FF30A000FF30A10065
:10018000FF30A20008000030A0000030A1000030C5
:10019000A2000800A01BCD28DA28A920DA20A9286F
:1001A000A101A201A301A01BD728E6208328A92032
:1001B000E620A928A4000310A00CA10CA20CA30CFB
:1001C000A40BDB280800A101A201A301A4000310D5
:1001D000A30DA20DA10DA00D0318BC28A40BE728A8
:1001E0000800A01BFF28A008031DAE282108A000BE
:1001F0002208A1002308A200A01BAE280800200AA4
:10020000031DB5282108A0002208A1002308A20090
:10021000A01FB5280800A008031DBC282108A000C5
:100220002208A1002308A20008002208A300210838
:10023000A2002008A100A001A11BA0030800220821
:10024000A3002108A2002008A100A0010800A0012D
:10025000A10100380319080003100018A007A00C22
:10026000A10C8018A007A00CA10C0019A007A00CDD
:10027000A10C8019A007A00CA10C001AA007A00CCB
:10028000A10C801AA007A00CA10C001BA007A00CB9
:10029000A10C801BA007A00CA10C0800801F27291F
:1002A0008009800A27218009800A9728A400840AEF
:1002B00027212108A3002008A200840324084E213E
:1002C0002208A1070318A00A2308A200080020089A
:1002D000A20021084E212108A6002008A50022081E
:1002E0005621A401A51BA403243084004628A400A1
:1002F000840A27212108A3002008A20084032408DF
:1003000027212208A1070318A00A2308A200080039
:100310002008A200210827212108A6002008A50006
:1003200022087721A401A51BA403243084004628B9
:100330000008A200840A0008A3002208230403196D
:10034000AB29A21BAB29A01BAB290310A30DA20D47
:10035000A10DA00DA1292208AD29A200A3012430DE
:1003600084002C20A5010830A000263084002C2019
:10037000A001A1010310A20CA30C223084003E2096
:100380002008240203190310A50D2518CA292230BC
:1003900084005620A60BBA292508A00008002108D1
:1003A000A3002008A2003E20801BDC29223084000C
:1003B0006F20031CBC280800223084006F20031823
:1003C000C32808002108A3002008A2003E20801BAB
:1003D000EF29223084007F20031CAE280800223041
:1003E00084007F200318B52808000730A0001930CA
:1003F00084002C200030A0009F3084002C2071301D
:10040000A0008F3084002C20813084008012801165
:100410008130840000148014001500100011252A7A
:100420002008FF0021040319A10A2108003C8100D3
:100430000318FF030B118B167E100800FF008101CB
:100440001A2AFF01003C81001A2A8312901010160C
:100450009016382A8E018F0110140C1008000F0816
:10046000A0000E08A1000F082002031D2F2A08007B
:10047000831283128C13592A83169B00572A8316E2
:100480001C1483161A08572A83161B08572A83162A
:100490009B0A572A83169B03572A83169B07572AC2
:1004A0003F228000840A4722A003031D502A8312A2
:1004B00008008312602AFF30A000FF30A10008006E
:1004C00083161F169F161F17892AA000203084004C
:1004D00083129F011F140018732A83161F147C2295
:1004E00083161F10792A1F1583169F147C228316EA
:1004F0009F108312A00008000A30FF3E031D7D2AD2
:1005000083129F149F18822A83121E0883121F10C1
:1005100008008312BB2AA200223084002008272171
:100520002108A20020084D223F22A30047223F229B
:10053000A4002408A1002308A0002208A20021088A
:10054000A4002008A300FF30A00022308400532024
:1005500023308400200827212108A6002008A500B8
:10056000223084001D2024308400200827212530DB
:1005700084003E2008008316051185129501831220
:100580008312CB251A263D260030A00020083C22ED
:100590000830A0002C3084005022B40185122A2299
:1005A0005F225B22FF30A400243084006C20031DF6
:1005B000C42A0F08A0000130E3202E3084006C20F4
:1005C0000318CD2A1C26031CD12A3608A900350899
:1005D000A8002F222A22353084002F20B40A34307C
:1005E00084001D200330A400243084006C200318F4
:1005F000FA2AD12A353084002020283084003E2079
:10060000353084002F207D26CB258D26B401BB01FB
:10061000BC012F08BD00FF30A000FF30A100373023
:1006200084002F205F22E030A00020085F221030DD
:10063000A0002D1CA00A20085F223E26031D292BA6
:100640003E26031D292B0D30A00020083C223F220E
:10065000A00020085F224E3084002C202830840027
:100660002C203030A0004F3084002C200C30A00013
:1006700028308400200827210B214F3084003B20A4
:100680004F3084002C2020083C223F22A0003E3026
:1006900084002C2047220B30A000503084005022D0
:1006A0000830A0005208AD215C3084002C200830B6
:1006B000A0005108AD21513084002C206023762BFE
:1006C000D701A0016623571F622B080057081F3966
:1006D000A03E840020088000D70A080020095707A0
:1006E0001F39A03E84000008A00008000F08A000E9
:1006F0003D3084006C200318862D1C26031C762BAD
:10070000B41F882B2F222A22393084003E20A92BA7
:100710002F222A22393084002F20353084005620A1
:10072000A01BA220283084002F20393084002020F4
:100730000130E420353084005620A01BA220283050
:1007400084006F203930840020200318A92BB417AF
:10075000762B353084002F200330E4202C18B22B68
:1007600020085F22B413353084001D2023213B3044
:1007700084003E203B3084002F20341B1D2CDE25BE
:100780007D265C252C18C62B20085F223F08C90057
:10079000DC234A3084001D20323084006C20031C8E
:1007A000D42B323084001D204A3084002C202C1899
:1007B000DB2B20085F22762B3B3084002020013089
:1007C000A400F430A500243084006F200318052C09
:1007D000353084002020373084006F200318FA2B36
:1007E000373084002F20B401FF30A0004A3084004D
:1007F0002C200800B40A343084001D200530A400E9
:10080000243084006C20031CF42BB4013417B7018E
:10081000B801493084001D20553084006C20031C31
:10082000122CB001DD01DE01DF01DA01DB01FF3056
:10083000A000583084002C2008008516B41E242CFB
:100840004B1D2E2C13262E2CDE25353084001D202A
:10085000303084006C20031C2E2CB41633308400FE
:100860001D2035308400200877210330A40000309B
:10087000A500243084006F20031C422C0330A0000C
:100880000030A100283084002F2035308400202043
:10089000283084005620393084002F2037308400DF
:1008A0002020353084003E20373084002F20A226BF
:1008B0005C252C185D2C20085F2235308400202018
:1008C0000330E420563084002C2041308400202066
:1008D0000330D1206623A801A9010030A0002A30EE
:1008E00084002C206E231921283084003E202830DB
:1008F00084002F202A3084001D20A00A0530A40087
:10090000243084006C20031C6F2C283084002020AD
:100910000530D1205E3084002C2028308400202037
:100920005A3084005620F120603084002C20A01B17
:10093000A0205D3084002C202908DB002808DA0084
:100940000830A0004F3084003B2020083C227F303C
:10095000A0005E3084005320523084006C20031CC1
:10096000B42C523084001D205E3084003B20862051
:100970005C308400200827210530E42028308400E2
:100980002C205D3084001D20513084002008272158
:100990000530E42003308B222830840020082721F2
:1009A0000630DA209720283084002F205830840029
:1009B000202028308400CF21583084002F20503050
:1009C0008400200827210A30A400243084006C20F1
:1009D0000318EC2C0A30A0004A3084002C205D3033
:1009E00084001D20533084006C20031C052D4A30E8
:1009F00084001D20543084006C20031C022D5430D0
:100A000084001D204A3084002C20373084001D20B3
:100A10002F3084006C20031C152D2F3084005320B0
:100A2000373084002F20F030B4053B308400202084
:100A30000330A400E830A500243084006F200318A0
:100A4000312D493084001D203F3084005320A01BED
:100A5000A0200930A400243084006C200318341630
:100A6000382D341A382D4E3084001D205025382D55
:100A7000B41ACE25FF30A000CB1B412D4A30840094
:100A80001D202C18452D20085F222F22393084008C
:100A90006F20031C452D85122C1D762B1026762BDE
:100AA00020083C222830A00020084D223F22A00030
:100AB0004A3084002C2008002D3084001D20043092
:100AC000A400243084006C200318802D20088A00A4
:100AD00005308A060A068A06703E03188A0A8200D2
:100AE000742D782D7E2D7F2D3F3084001D20080031
:100AF0004130840020200330D12008000800080085
:100B00002008593E84000008A000080085160D2624
:100B10004130A0008F3084002C20B501B6014A304E
:100B200084001D20AC1C962DE530A0000330DA2097
:100B30004A3084002C200515353084002020A10A7D
:100B4000031DA32DA00A353084002F200330A400FC
:100B5000243084006C20AC1CB22D0A30A400243058
:100B600084006C2003180028013084001D201F30F1
:100B7000A0054A3084006C20031CB42D05110130FF
:100B800084001D201F30A0054A3084006C2003180B
:100B9000BF2D05159C2DCA01CC010D2EEF254C3023
:100BA00084002C204B180800CC08031908000515F8
:100BB0004B14CB140830DA2010220800EF25353012
:100BC00084002008772110220515CB010800A00819
:100BD0000319080010220515CB14CB170800183094
:100BE000A00020083C224A3084001D200F308B22B8
:100BF00008004B1C0D2ECB18062ECB144B19012EC2
:100C000005154C08FF3C81008B160800CB10CB1358
:100C100005114C0881008B160800CB010511080056
:100C20004B15051108004B1D08004B11CB1C08008B
:100C300005150800851608000314051A0310CD0CCD
:100C40000318282E4D10E0304D0203184D140800F3
:100C50004D1410304D02031C4D10031008000314F6
:100C6000051A0310A001A00D20085F220B30A00080
:100C700020085F2220085F2208000800003065225B
:100C80002321283084002F200C30A00020083C2293
:100C90003F22A0002A3084002C200E30A000200823
:100CA0003C22AB013F22A000FF30A400243084008E
:100CB0006C2003196E2E2321283084005620F12049
:100CC000A01BA0202A3084006C20031C6A2EAB0AD3
:100CD0004722522E2B08A0000311080008003E26D0
:100CE00020085F22283084001D2020085F22293040
:100CF00084001D2020085F220800BF01C001C1013F
:100D0000C101C201C301C830A000232135308400D5
:100D100098213F3084002C200800313084001D20B1
:100D20000130E320473084002C20313084001D2026
:100D300031308400200827210430E420483084002A
:100D40002C2008000630A0004730A100AE30A200E1
:100D50002830840034203530840020203F30840047
:100D6000882183200530CA20F120A5202830840066
:100D70004620F120453084002F20473084001D207C
:100D800045308400200856210530CA203F308400B9
:100D90003E203F3084002F20353084002020413019
:100DA000840067210730CA20F1203F3084003E20B4
:100DB0003F3084002F203E3084001D204A308400C4
:100DC000200827212321CB1FF62E4630A0003E30DD
:100DD0008400200827212321283084002F203E3042
:100DE00084001D202321283084003E208320A2205F
:100DF0003F3084003E203F3084002F204830840064
:100E00001D2045308400200856210330CA2043307D
:100E100084002F20413084003E20413084002F2068
:020E20000800C8
:02400E00D430AC
:10420000000001000E001100FF0023006400820086
:084218000500010048006D00E3
:0242200092000A
:1042300014001E002D003C0044005500660077006D
:1042400088009900AA00BB00CC00DD00EE00FF0052
:0E42500005002D0055007D00A500CD00F500F5
:1042600096004600320032001400320000000000C8
:1042700000004600640064009600640032003200D2
:10428000140032000000000000003C005A006400EE
:1042900096008C0032003200140032000000000052
:0842A000000032005000640030
:00000001FF
